:100000000C9449010C9466010C9466010C946601F1
:100010000C9466010C9466010C9466010C946601C4
:100020000C9466010C9466010C9466010C946601B4
:100030000C9466010C9466010C9469050C9466019D
:100040000C9466010C9466010C94A9010C94E501D2
:100050000C9466010C9466010C9466010C94660184
:100060000C9466010C9466012C003A00456E644FB6
:1000700066536F61702100312E304230310054617F
:100080006B74676562657220005368757444005A2A
:100090007572636B0020202020202000205368759B
:1000A00074440020004572726F7200536875746466
:1000B000004E6F726D6C005072536530005072507C
:1000C00075420020202020202020202020200020F9
:1000D0002020202020202020202050726F677200D6
:1000E0004572726F720053687574640050726F6766
:1000F00072004E6D535A74004E6D566B7A004E6D01
:10010000537672004E6D556872002020202020200A
:1001100000204E6F726D6C00200050726F6772008D
:100120004E6F726D6C00202020002D0044002D00C9
:1001300047002D0045002D002D002D002D0045000D
:100140002D005379735374617475732020496E695F
:10015000742000456E7465722068696C66742100B5
:10016000312E304230310054616B746765626572C4
:10017000200055702F446F776E202020205A757212
:10018000636B002020202020204E6D535A740045C0
:1001900072726F72005A7572636B0053746E64658D
:1001A000004D696E74650020202020202020202032
:1001B0002020002020202020204E6D535A7400550E
:1001C000702F446F776E202020205A7572636B0069
:1001D000204E6D566B7A0020202020202000457292
:1001E000726F720053746F7020005A7572636B00E7
:1001F0005374617274004572726F720053764E755B
:100200006C005376537274004572726F72005A75A7
:1002100072636B0053764E756C00537653727400A4
:100220004E6D537672004572726F720053746F7028
:1002300020005A7572636B00537461727400202041
:100240002020202000204E6D556872002000507242
:10025000536530005A7572636B00202020202020E7
:1002600000205072536530002020202020202020C4
:1002700020200055702F446F776E202020205A7563
:1002800072636B002053656B2020205072507542C2
:10029000000011241FBECFEFD4E0DEBFCDBF11E0C0
:1002A000A0E0B1E0E4EBFFE102C005900D92A230C6
:1002B000B107D9F711E0A2E0B1E001C01D92A83A60
:1002C000B107E1F70E9468010C94D90F0C9400006B
:1002D0001F930E942C090E94500578940E941F09C8
:1002E0000E94FF08182F113011F40E94A5080E94E7
:1002F000CD08182F8230B8F30E948308882399F321
:100300000E94730880E090E01F9108958BB19927B7
:100310009695879596958795809590958170907024
:1003200008959091840180918501981730F0909103
:10033000840180918501981B06C090918401809171
:100340008501981B905C953110F05A9A08955A983F
:1003500008951F920F920FB60F9211242F933F937F
:100360004F935F936F937F938F939F93AF93BF93BD
:10037000EF93FF939091C0002091C600E09184011B
:10038000EF5FEF7380918501E81711F482E008C0F8
:10039000892F8871E0938401FF27EE5BFE4F208355
:1003A000809386010E949101FF91EF91BF91AF91DF
:1003B0009F918F917F916F915F914F913F912F917D
:1003C0000F900FBE0F901F9018951F920F920FB6AF
:1003D0000F9211248F939F93EF93FF93909182013B
:1003E00080918301981769F0E0918301EF5FEF73CB
:1003F000E0938301FF27EE5FFE4F80818093C6006C
:1004000005C08091C1008F7D8093C100FF91EF9165
:100410009F918F910F900FBE0F901F901895109283
:10042000820110928301109284011092850198E953
:100430009093C1008093C4005A98529A08951F93D4
:100440009091840180918501981719F480E091E0E2
:1004500013C0E0918501EF5FEF73E0938501FF2703
:10046000EE5BFE4F10810E949101809186019927D9
:10047000982F8827810F911D1F91089590918401D5
:100480008091850120E030E0981711F021E030E004
:10049000C90108950F931F93909184018091850164
:1004A0009817D1F3009185010F5F0F7300938501B9
:1004B0000E94910111270E5B1E4FF8018081992740
:1004C0001F910F910895282F909182019F5F9F7334
:1004D000809183019817E1F3E92FFF27EE5FFE4F2C
:1004E0002083909382018091C10080628093C1003B
:1004F0000895CF93DF93EC0103C021960E9463021D
:1005000088818823D1F7DF91CF9108952F923F9270
:100510004F925F926F927F928F929F92AF92BF9213
:10052000CF92DF92EF92FF920F931F93CF93DF93BF
:10053000CDB7DEB761970FB6F894DEBF0FBECDBF63
:100540008F87798B688B4A01442455241E861D862B
:1005500001C1262D332720FF46C1872D80538A30C5
:1005600008F452C187E6871554F195E679160CF028
:100570004CC0E3E57E1609F461C0E715ACF0FBE280
:100580007F1609F441C1F7154CF020E2721609F408
:100590003BC133E2731609F024C136C1872D8D5259
:1005A000823008F01EC130C183E6781689F18715C4
:1005B0000CF456C098E5791609F013C11FC0E0E7A6
:1005C0007E16D1F0E71564F0FCE67F16D9F08FE6D1
:1005D000781609F469C099E6791609F002C140C09D
:1005E000E5E77E1609F463C0F8E77F1639F023E7E4
:1005F000721609F0F6C013C068E7762E50E1452E5A
:10060000512C55C034E0632AFFC04FE3A42E9AC09A
:10061000F401A08022E030E0820E931E93C0F4012A
:10062000A080B18044245524F50104C00894411CE5
:10063000511C319680818823C9F7FBC0F401A0804A
:10064000B1809501F50101C0319684918823E1F7CD
:1006500082E090E0880E991E2F01421A530A7FC053
:1006600022FF08C0F40180819181A281B38124E03E
:1006700030E009C0F40180819181AA2797FDA095FF
:10068000BA2F22E030E0820E931E5C016D01B7FFAD
:1006900023C032E0632AD094C094B094A094A11CEB
:1006A000B11CC11CD11C18C038E0432E512C22FFB4
:1006B00008C0F40180819181A281B38124E030E0FF
:1006C00007C0F40180819181AA27BB2722E030E096
:1006D000820E931E5C016D01860175011E01089456
:1006E000211C311C5201CC24DD24C801B701A60114
:1006F00095010E948F0F6A301CF0670D615201C096
:10070000605DF10161931F01C801B701A601950168
:100710000E948F0F79018A0121153105410551058C
:1007200021F7AA24BB24650161FE09C08DE20E9465
:1007300063022D853E852F5F3F4F3E872D8733E631
:10074000731651F48A2D0E9463028D859E85019651
:100750009E878D87662458C093E5791691F48501AC
:10076000720106C0F80184910E9463020F5F1F4F5F
:100770000894E108F108FFEFEF16FFEFFF0691F78D
:1007800013C033E7731611F081011DC0750182019A
:1007900005C0F70181917F010E9463020150104062
:1007A000FFEF0F3F1F07A9F72D853E85240D351D4F
:1007B0003E872D872FEF422E522ECCCFF80182910B
:1007C0008F010E946302CE01019608171907B1F745
:1007D000281A390A2D853E85220D331D3E872D8727
:1007E000B9CF872DB0CF95E2791631F49AE0492E32
:1007F000512C81E0682E08C0872D0E946302ED8590
:10080000FE853196FE87ED87888999890196FF8557
:10081000F13031F4E889F989998B888B749005C09F
:10082000E889F9897080998B888B772009F091CEBF
:1008300005C022E030E0820E931EA8CF8D859E85F4
:1008400061960FB6F894DEBF0FBECDBFDF91CF919A
:100850001F910F91FF90EF90DF90CF90BF90AF90DE
:100860009F908F907F906F905F904F903F902F90D0
:100870000895CF93DF93CDB7DEB722970FB6F894E4
:10088000DEBF0FBECDBFFE01379661917191FA8335
:10089000E983AF0181E00E94860222960FB6F894A8
:1008A000DEBF0FBECDBFDF91CF910895CF93DF9311
:1008B000CDB7DEB722970FB6F894DEBF0FBECDBF1F
:1008C000FE01379661917191FA83E983AF0180E06F
:1008D0000E94860222960FB6F894DEBF0FBECDBFEF
:1008E000DF91CF910895FC01892B59F1808191818D
:1008F000A281B3810097A105B10519F14F5F5F4F48
:100900006F4F7F4F4F3F2FEF52072FEF62072FE3BD
:100910007207B8F4840F951FA61FB71F80839183B9
:10092000A283B3830097A105B10541F481E090E073
:10093000A0E0B0E080839183A283B38380E090E065
:1009400008958FEF9FEF0895FC01108211821282AB
:1009500013820895EF92FF920F931F93CF93DF932B
:10096000EC017A018B01411551056105710531F4E6
:1009700091E0E92EF12C012D112D1BC04E3F8FEF80
:1009800058078FEF68078FE7780748F08DEFE82E5C
:100990008FEFF82E8FEF082F8FE7182F05C0495ED5
:1009A00053406040704028F00894E11CF11C011D88
:1009B000111D0E945D056E0D7F1D801F911F6883B4
:1009C00079838A839B83611571058105910541F4C3
:1009D00081E090E0A0E0B0E088839983AA83BB83A4
:1009E000DF91CF911F910F91FF90EF900895CF93DA
:1009F000DF93EC0188819981AA81BB810097A105D1
:100A0000B10519F48FEF9FEF27C00E945D05288183
:100A100039814A815B81621773078407950750F417
:100A2000261B370B480B590B2E5F3F4F4F4F5F472D
:100A300088F009C0621B730B840B950B6E5F7F4FB0
:100A40008F4F9F4738F4188219821A821B8280E0E8
:100A500090E002C081E090E0DF91CF910895CF93C4
:100A6000DF93CDB7DEB724970FB6F894DEBF0FBE85
:100A7000CDBFAA27BB27AC01BD01CE0101960E94C4
:100A8000AA04CE0101960E94F7048823D1F7249688
:100A90000FB6F894DEBF0FBECDBFDF91CF910895A2
:100AA00084B5826084BD83E085BD8AEF87BDEEE6B4
:100AB000F0E080818260808308958FB7F8948FBFC3
:100AC00060918701709188018091890190918A01DC
:100AD00008951F920F920FB60F9211241F932F9318
:100AE0003F934F935F936F937F938F939F93AF93B6
:100AF000BF93EF93FF938091870190918801A0911C
:100B00008901B0918A010196A11DB11D80938701D1
:100B100090938801A0938901B0938A010E94CA062C
:100B200080910001815080930001882391F41AE0A4
:100B3000109300010E94BD070E94CB068091010125
:100B4000815080930101882321F4109301010E94B8
:100B50008807FF91EF91BF91AF919F918F917F9106
:100B60006F915F914F913F912F911F910F900FBE09
:100B70000F901F9018958115910511F00197F1F7CD
:100B800008952BB12F7087FD2068992786FD20647A
:100B900085FD206284FD20612BB95B9A5B982F70E4
:100BA00083FD206882FD206481FD206280FD20613C
:100BB0002BB95B9A5B9880E892E08115910511F062
:100BC0000197F1F708955A9881E00E94C10580E1EC
:100BD00090E48115910511F00197F1F70895CF93F5
:100BE000DF93EC015A9A03C021960E94C1058881C7
:100BF0008823D1F7DF91CF910895CF93DF93EC0154
:100C00005A9A03C00E94C1052196FE01849188234F
:100C1000C9F7DF91CF9108955A9A0E94C1050895AE
:100C20005A98662349F0613011F4805C05C0623047
:100C300011F4805F01C0805B80680E94C105089547
:100C4000FF920F931F93F82E062F142F0E94100669
:100C500003C080E20E940C061150D8F7602F8F2D40
:100C60000E9410061F910F91FF900895DF92EF925E
:100C7000FF920F931F93CF93DF93CDB7DEB72B97E0
:100C80000FB6F894DEBF0FBECDBF7C01D62E4BE071
:100C900050E060E270E08E010F5F1F4FC8010E94BC
:100CA000430F4AE050E0BE016A5F7F4FC7010E94D8
:100CB0004A0FFC0101900020E9F73197E81B0E0F65
:100CC000111D0D191109C80105960E94EF052B96FB
:100CD0000FB6F894DEBF0FBECDBFDF91CF911F914D
:100CE0000F91FF90EF90DF9008951F93182F529A65
:100CF000539A8AB1806F8AB95A985B9880E09AEFCC
:100D00008115910511F00197F1F75C9A5D9A5B9A54
:100D10005B9880E29EE48115910511F00197F1F74F
:100D20005B9A5B9880E892E08115910511F001973C
:100D3000F1F75B9A5B9880E892E08115910511F0DC
:100D40000197F1F75C985B9A5B9880E892E08115D7
:100D5000910511F00197F1F788E20E94C10588E042
:100D60000E94C1050E94E30586E00E94C10586E05D
:100D70000E94C105812F0E94C1051F91089588B16D
:100D8000807F88B987B18F6087B988B1896088B959
:100D900008950895089508950895282F3FB7F89469
:100DA00080938B01882379F080918E0190918F013F
:100DB00090938D0180938C01233028F080919301D2
:100DC0008170809392013FBF08958FB7F8948FBFD1
:100DD00080918B01992708952FB7F89490938F01F4
:100DE00080938E012FBF08958FB7F8948FBF8091A5
:100DF0008E0190918F0108952FB7F89490939101EF
:100E0000809390012FBF08958FB7F8948FBF809182
:100E100090019091910108959FB7F8948093930168
:100E20009FBF08958FB7F8948FBF80919301992742
:100E300008959FB7F894809394019FBF08958FB74A
:100E4000F8948FBF809194019927089540918B0168
:100E5000442309F443C080918C0190918D01019746
:100E600090938D0180938C01892B51F480918E0198
:100E700090918F0190938D0180938C0141984298BD
:100E800020918C0130918D01809190019091910180
:100E900028173907E1F580919201882329F481E030
:100EA00080939201429A03C010929201419A43307A
:100EB00070F1809193018F5F809393018C3338F0B0
:100EC00010929301809194018F5F8093940180919F
:100ED00094018831E0F0109294010895419902C084
:100EE000429B15C080918C0190918D010197909348
:100EF0008D0180938C01892B51F480918E0190910A
:100F00008F0190938D0180938C01419842980895B0
:100F10000E942607089585B18C6385B9E5E9F1E063
:100F2000ADE9B1E0119211921D9281E0ED39F8071F
:100F3000C9F708959FB7F8949FBFEDE9F1E0E80F76
:100F4000F11D808199270895E82F8FB7F8948FBFFE
:100F5000FF27EE0FFF1FEB56FE4F80819181089512
:100F60009FB7F894E82FFF27E356FE4F8081882330
:100F700011F0806880839FBF08951A9918C08091EE
:100F80009501909196010196909396018093950119
:100F90008530910521F480919D01816005C0C29743
:100FA00061F480919D01826080939D0106C0109242
:100FB00096011092950110929D011B9918C0809185
:100FC00097019091980101969093980180939701D1
:100FD0008530910521F480919E01816005C0C29702
:100FE00061F480919E01826080939E0106C0109200
:100FF00098011092970110929E011C9918C080913F
:10100000990190919A01019690939A018093990188
:101010008530910521F480919F01816005C0C297C0
:1010200061F480919F01826080939F0106C01092BD
:101030009A011092990110929F011D9918C08091F8
:101040009B0190919C01019690939C0180939B0140
:101050008530910521F48091A001816005C0C2977F
:1010600061F48091A00182608093A00108951092A4
:101070009C0110929B011092A00108950895FF9287
:101080000F931F93182FF62E042F82E00E949A07C9
:1010900081FF05C08AEF90E00E942F0505C0181659
:1010A0003CF482E00E94B0071F5F011708F41F2D77
:1010B00083E00E949A0781FF05C08AEF90E00E94BA
:1010C0002F0505C018164CF483E00E94B00711509C
:1010D000011710F01F1508F4102F812F99271F9169
:1010E0000F91FF90089580E00E94CD060E94EB0BC7
:1010F0000E94690980E00E949A071816CCF780E0E8
:101100000E94B007F5CF1F9310E0812F0E94190AAB
:1011100041E060E0812F0E943F08182F80E00E948C
:101120009A07181634F480E00E94B007812F99279F
:101130000AC081E00E949A0718163CF781E00E94DD
:10114000B00780E090E01F9108951F9310E0812F79
:101150000E947E0943E060E0812F0E943F08182F23
:1011600080E00E949A07181694F780E00E94B0076A
:10117000112319F40E94DB0EEACF113019F40E94FA
:10118000B50EE5CF123019F480E090E004C01330C2
:10119000F1F682E090E01F9108951F9310E0812FF7
:1011A0000E94540A45E060E0812F0E943F08182FFA
:1011B00080E00E949A07181694F780E00E94B0071A
:1011C000112319F40E944D0DEACF113019F40E9439
:1011D000190DE5CF123019F40E94F60CE0CF133050
:1011E00019F40E94880CDBCF143019F481E090E0F0
:1011F00004C01530A1F682E090E01F9108950F938E
:101200001F930E94E90A082F10E0813009F011E0D5
:10121000602F812F0E94AA0941E060E0812F0E9487
:101220003F08182F80E00E949A0718168CF780E07C
:101230000E94B007812F99271F910F9108950E9456
:10124000040A80E00E949A071816DCF780E00E94EA
:10125000B00780E090E008950E94BF060E948B07CF
:101260000E94A80A08950895EF92FF921F93182FE5
:101270006AE00E94700FE82E62E099270E9436060D
:1012800088E690E00E94FD058AE0E89E7001112446
:101290001E1961E0812F99270E9436061F91FF9049
:1012A000EF9008950F931F93062F992762E08C59B2
:1012B0009F4F0E9436068AE690E00E94FD051127A6
:1012C00062E0C8018C599F4F0E9436061F910F9112
:1012D000089560E080E00E9410068EE790E00E9492
:1012E000FD0587E790E00E94FD0561E080E00E9437
:1012F00010068CE690E00E94FD0508951F93182FBC
:1013000060E080E00E9410068FEC90E00E94FD05F6
:1013100061E080E00E94100683EC90E00E94FD05F1
:10132000112319F48DEB90E011C0113019F487EB03
:1013300090E00CC0123019F481EB90E007C013303C
:1013400019F48BEA90E002C085EA90E00E94FD0566
:101350001F9108950F931F93CF93DF93082F162F9C
:1013600060E080E00E94100682E491E00E94FD05AA
:1013700061E080E00E94100680E491E00E94FD059B
:10138000C12FDD27C6FF03C08EE391E002C08CE3CE
:1013900091E00E94FD058AE391E00E94FD0588E34B
:1013A00091E00E94FD0586E391E00E94FD05C2FFE9
:1013B00003C084E391E002C082E391E00E94FD0556
:1013C000C1FF03C080E391E002C08EE291E00E9481
:1013D000FD05C0FF03C08CE291E002C08AE291E00B
:1013E0000E94FD0586E291E00E94FD05002319F4AC
:1013F00080E291E002C08AE191E00E94FD05DF9168
:10140000CF911F910F91089560E080E00E94100637
:1014100087E691E00E94FD0580E691E00E94FD05CF
:1014200061E080E00E94100683E591E00E94FD05E6
:1014300008950F931F93082F60E080E00E9410062C
:101440000E94C10A182F0E94C80A612F0E945209E7
:1014500083EA90E00E94FD050E94BA0A0E943409C6
:101460008CE990E00E94FD0561E085E00E94100695
:1014700085E990E00E94FD05002319F48FE890E0D3
:1014800002C089E890E00E94FD0561E080E00E94D2
:1014900010060E941207182F0E941F07612F0E943A
:1014A00052091F910F9108950F931F93082F60E029
:1014B00080E00E9410060E94C10A182F0E94C80AEC
:1014C000612F0E94520988E191E00E94FD050E946F
:1014D000BA0A0E94340981E191E00E94FD0561E0B1
:1014E00085E00E9410068AE091E00E94FD0500233D
:1014F00019F484E091E01BC0013019F48EEF90E004
:1015000016C0023019F488EF90E011C0033019F4CE
:1015100082EF90E00CC0043019F48CEE90E007C02C
:10152000053019F486EE90E002C080EE90E00E9453
:10153000FD0561E080E00E9410060E941207182F4E
:101540000E941F07612F0E9452091F910F91089559
:101550008CE00E94750608958093A1010895809102
:10156000A101992708958093A70108958091A7016B
:10157000992708958091A201992708958093A30146
:1015800008958091A301992708958093A401089557
:101590008091A401992708958093A50108958091D1
:1015A000A501992708958093A60108958091A60129
:1015B000992708958A3008F48AE08093A201682F61
:1015C000772780E797E10E947C0FCB010E94EC0611
:1015D00008952F923F924F925F926F927F928F92D7
:1015E0009F92AF92BF92CF92DF92EF92FF920F93B2
:1015F0001F93CF93DF93CDE0D0E0DE010E94C50FB3
:10160000802D99278093A70104E010E075E0E72E74
:1016100070E0F72E69E0C62E60E0D62E5AE0A52EC7
:1016200050E0B52E4BE0842E40E0942E3CE0632E3B
:1016300030E0732E26E0422E20E0522E97E0292E35
:1016400090E0392E8A3F08F45FC01092A70181E034
:101650008093A10184E68093A2011092A3011092CD
:10166000A4011092A5011092A6018CE390E00E94C3
:10167000EC068AE090E00E94FC0680E00E940C07E5
:1016800087E10E9419078091A701DE01082E0E94C0
:10169000CD0F8091A101D801082E0E94CD0F80911D
:1016A000A201D701082E0E94CD0F8091A301D6017F
:1016B000082E0E94CD0F8091A401D501082E0E9412
:1016C000CD0F8091A501D401082E0E94CD0F8091ED
:1016D000A601D301082E0E94CD0F0E940407D2015B
:1016E000082E0E94CD0F0E941207D101082E0E94E1
:1016F000CD0F0E941F07A8E0B0E0082E0E94CD0F7A
:101700008091A101846047C0D8010E94C50F802D3F
:101710008093A101D7010E94C50F802D9927682FC2
:101720008093A201D6010E94C50F802D8093A30152
:10173000D5010E94C50F802D8093A401D4010E9481
:10174000C50F802D8093A501D3010E94C50F802D68
:101750008093A601772780E797E10E947C0FCB0159
:101760000E94EC06D2010E94C50F802D99270E948D
:10177000FC06D1010E94C50F802D0E940C07A8E035
:10178000B0E00E94C50F802D0E9419078091A10131
:10179000882321F082608093A10107C081E08093BB
:1017A000A101D801082E0E94CD0F8091A101992797
:1017B000DF91CF911F910F91FF90EF90DF90CF902D
:1017C000BF90AF909F908F907F906F905F904F9061
:1017D0003F902F9008958091A10180748093A10182
:1017E0008091A701ADE0B0E0082E0E94CD0F80915E
:1017F000A101A4E0B0E0082E0E94CD0F8091A201CB
:10180000A5E0B0E0082E0E94CD0F8091A301A9E0D1
:10181000B0E0082E0E94CD0F8091A401AAE0B0E0B4
:10182000082E0E94CD0F8091A501ABE0B0E0082EFC
:101830000E94CD0F8091A601ACE0B0E0082E0E947E
:10184000CD0F0E940407A6E0B0E0082E0E94CD0F45
:101850000E941207A7E0B0E0082E0E94CD0F0E9460
:101860001F07A8E0B0E0082E0E94CD0F089508954C
:10187000EF92FF920F931F93182F882319F0EE24F5
:10188000FF2406C00E94C10AE82E0E94C80AF82E52
:1018900000E02F2D4E2D602F812F0E94E60D41E09C
:1018A00060E0802F0E943F08082F80E00E949A0786
:1018B00018160CF580E00E94B007002321F583E0A4
:1018C0000E94CD062F2D4E2D62E0812F0E94E60D45
:1018D0000E941F078F1521F40E9412078E1541F0F8
:1018E00080E00E949A0718166CF780E00E94B0070B
:1018F00080E00E94CD0681E00E949A0718164CF6FF
:1019000081E00E94B0071F910F91FF90EF90089522
:10191000FF920F931F93FF248F2D0E949A0D42E098
:1019200060E08F2D0E943F08F82E80E00E949A0709
:1019300018160CF04EC080E00E94B007FF2049F559
:101940000E94C10A182F0E94C80A082F602F812FF9
:101950000E947F0D4BE360E0812F0E943F08182F0B
:1019600080E00E949A07181634F081E00E949A07DE
:10197000181664F72BC080E00E94B007812F0E94E8
:10198000BE0A27C080E00E94B007812F0E94C50ACE
:1019900020C081E0F81631F50E94C10A082F0E948C
:1019A000C80A182F612F802F0E947F0D47E160E049
:1019B000812F0E943F08182F80E00E949A07181676
:1019C0000CF381E00E949A07181664F781E00E94E8
:1019D000B00781E00E949A0718160CF09DCF81E0B5
:1019E0000E94B0071F910F91FF9008951F930E94CE
:1019F000BA0A182F812F0E94CB0D47E76AE0812F8A
:101A00000E943F08182F80E00E949A0718163CF4A5
:101A100080E00E94B007812F0E94DA0A08C081E0AE
:101A20000E949A07181634F781E00E94B0071F91B0
:101A30000895FF920F931F930E94E305FF248F2DBB
:101A40000E94330E42E060E08F2D0E943F08F82E86
:101A500080E00E949A071816A4F480E00E94B00764
:101A600081E08F15B0F00E94F4068C0184E190E0D3
:101A70000E94EC068F2D0E94380C802F99270E941F
:101A8000EC0681E00E949A071816CCF681E00E94CD
:101A9000B0071F910F91FF9008951F9310E0812FC1
:101AA0000E94700E41E060E0812F0E943F08182FD5
:101AB00080E00E949A071816B4F480E00E94B007F4
:101AC0001123C9F483E00E94CD0682E00E94700ECB
:101AD00080E00E949A071816C4F780E00E94B007C1
:101AE00080E00E94CD0681E00E949A071816BCF69D
:101AF00081E00E94B0071F910895089508950F9303
:101B00001F93182F062F60E080E00E941006612FBF
:101B1000802F0E94520983E891E00E94FD0561E058
:101B200080E00E94100682E791E00E94FD051F916F
:101B30000F9108950F931F93082F60E080E00E949B
:101B400010060E94C10A182F0E94C80A612F0E9425
:101B5000520983EB91E00E94FD0561E080E00E9464
:101B6000100687EA91E00E94FD05002319F481EA3E
:101B700091E00CC0013019F48BE991E007C002300C
:101B800019F485E991E002C08FE891E00E94FD051B
:101B90001F910F9108951F93182F60E080E00E941D
:101BA000100687ED91E00E94FD05812F0E94340907
:101BB00080ED91E00E94FD0561E080E00E9410064A
:101BC0008FEB91E00E94FD051F910895EF92FF9227
:101BD0000F931F93E82EF62E142F022F60E080E063
:101BE0000E941006612F802F0E94520960E08BE056
:101BF0000E941006EE2019F482E092E008C081E015
:101C0000E81619F48CEF91E002C086EF91E00E9493
:101C1000FD0561E080E00E9410060E941207182F67
:101C20000E941F07612F0E94520961E08BE00E9411
:101C30001006FF2019F480EF91E00EC081E0F81645
:101C400019F48AEE91E008C082E0F81619F484EEE7
:101C500091E002C08EED91E00E94FD051F910F9171
:101C6000FF90EF9008950F931F93082F60E080E09E
:101C70000E9410060E94C10A182F0E94C80A612FF4
:101C80000E94520960E08BE00E94100680E292E020
:101C90000E94FD0561E080E00E9410060E9412078C
:101CA000182F0E941F07612F0E94520961E08BE0EC
:101CB0000E941006002319F48AE192E00CC0013062
:101CC00019F484E192E007C0023019F48EE092E04A
:101CD00002C088E092E00E94FD051F910F910895D7
:101CE0000F931F93082F60E080E00E9410060E946F
:101CF000C10A182F0E94C80A612F0E9452098CE461
:101D000092E00E94FD050E94BA0A0E94340985E40F
:101D100092E00E94FD0561E085E00E9410068EE3DE
:101D200092E00E94FD05002319F488E392E00CC0C4
:101D3000013019F482E392E007C0023019F48CE21A
:101D400092E002C086E292E00E94FD0561E080E040
:101D50000E9410060E941207182F0E941F07612F71
:101D60000E9452091F910F9108951F9310E0812F37
:101D70000E94FF0E41E060E0812F0E943F08182F73
:101D800080E00E949A07181664F480E00E94B00771
:101D9000113079F480E00E940C0780E00E9419075E
:101DA00008C081E00E949A0718160CF781E00E9493
:101DB000B0071F9108951F930E940407182F812FC9
:101DC0000E942C0F43E165E0812F0E943F08182FED
:101DD00080E00E949A07181644F480E00E94B00741
:101DE000812F99270E94FC0608C081E00E949A0773
:101DF00018162CF781E00E94B0071F9108951F93D9
:101E0000182F60E080E00E94100688E692E00E94B1
:101E1000FD0581E692E00E94FD0561E085E00E94FB
:101E200010068AE592E00E94FD05112319F484E56D
:101E300092E002C08EE492E00E94FD0561E080E045
:101E40000E9410060E941207182F0E941F07612F80
:101E50000E9452091F9108951F93182F60E080E09F
:101E60000E941006812F0E94340984E892E00E94AB
:101E7000FD0561E080E00E94100683E792E00E9489
:101E8000FD051F910895DC0101C06D934150504044
:101E9000E0F70895FB019F01423074F0453264F48D
:101EA000642F77270E94B10F805D8A330CF0895D23
:101EB0008193CB010097A1F71082C9010C94600FA8
:101EC000DC01FC01672F71917723E1F7329704C0A1
:101ED0007C916D9370836291AE17BF07C8F308952C
:101EE000991B79E004C0991F961708F0961B881F6C
:101EF0007A95C9F78095089597FB092E07260AD091
:101F000077FD04D02ED006D000201AF4709561958C
:101F10007F4F0895F6F7909581959F4F0895A1E220
:101F20001A2EAA1BBB1BFD010DC0AA1FBB1FEE1F53
:101F3000FF1FA217B307E407F50720F0A21BB30B9E
:101F4000E40BF50B661F771F881F991F1A9469F71A
:101F500060957095809590959B01AC01BD01CF0176
:101F60000895AA1BBB1B51E107C0AA1FBB1FA617E0
:101F7000B70710F0A61BB70B881F991F5A95A9F732
:101F800080959095BC01CD010895F999FECFB2BD21
:101F9000A1BDF89A119600B40895F999FECFB2BD8B
:101FA000A1BD00BC11960FB6F894FA9AF99A0FBE2B
:041FB0000895FFCFC2
:021FB4000A0A17
:00000001FF
